:020000002728AF
:08000800922A820733343234DE
:1000100028340C3406340134820700341234253479
:1000200037345034623475348234820701340234F8
:100030000434083482075034613473342034820726
:1000400031343234353430343034303430340330B9
:10005000860085118316173085000030860008154C
:10006000831297012E309000E9202A21DF204721BA
:10007000BA21051E482852205A21051D6328051C57
:100080008128851CB02897010530A900A8103928BF
:10009000051D7028051CA628851CD5289701A810C9
:1000A000852139282122C330960045223522672236
:1000B0002C2215084039031D60284E309400622818
:1000C0004C3094000800A8186F28A814003089004C
:1000D000180896008122890A19089600812247286B
:1000E000A8187828A81402308900240896008122D4
:1000F00051281708003C03188028970318227928F4
:1001000008002908003C03188928A9037920083031
:100110009700240815209A00153019020318982812
:10012000980F9F28990A15301902031C9F289928B7
:10013000980AE0301802031C9F28990198019A0B35
:100140008C28DF20BA215A214721472879200830FE
:100150009700240A0339A400852118221822512867
:100160002908003C0318B828A90379200830970013
:10017000240815209A0019080319C528980318089F
:10018000FF3C031DCE289903CE2898031808FF3C96
:10019000031DCE28E0309800153099009A0BBB283B
:1001A000DF20BA215A2147214728792008309700BB
:1001B00024030339A40085211822182251282F3046
:1001C000A000843018070318A00AA1001908A0078E
:1001D00008009A0118221A080520A700013086009D
:1001E00086152708F0398607000086111822A70E09
:1001F0000130860086152708F03986070000861131
:100200009A0A1A08063C031DEA28080001308600F5
:100210000B290330860086152708F039860713223C
:10022000861106080F3986008615270EF0398607D5
:10023000132286110330860008008316F0308600F2
:100240008312861506088039861186158611031DCE
:1002500021290800003089007A2215089800890AAF
:100260007A2215089900890A7A221508A400153007
:100270001902031C4129E0301802031C412999018D
:10028000980104302402031C4629A4010800000040
:100290002122C230960045222008960045222108DE
:1002A00096004522AE3096004522FF30960045224A
:1002B0002C2208000230A700062111229A0100001A
:1002C0001A080C301A0784000008A70009219A0AAE
:1002D0001A08083C031D5F2900002030A7000921EF
:1002E00000004D30A700092100004830A700092177
:1002F00000007A30A700092100002030A700092162
:1003000000001408A700092108000230A7000621F8
:1003100011229A011A081A20A70009219A0A1A081C
:10032000043C031D8A292408033C031D9A2931300B
:10033000A70009219A011A0824071F20A7000921F4
:100340009A0A1A08033C031D9B2900002030A700CD
:10035000092100006B30A700092100004830A700E8
:10036000092100007A30A700092100002030A700F1
:100370000921080030308C008D008E008F00910024
:10038000920093002008A2002108FC3E0318A20A54
:10039000A3000E30A207230807390C209E000F3956
:1003A00092071E0E0F399107231CD8290530930799
:1003B0002308F8399E0022089F0003109F0C9E0C12
:1003C0009F0C9E0C9F0C9E0CEC2918309E07031866
:1003D0009F0AFC309F078C0A03301F02E830031984
:1003E0001E020318E529F9299C309E07031C9F0370
:1003F0008D0A00301F02643003191E020318F4290D
:10040000062AF6309E07031C9F038E0A00301F0247
:100410000A3003191E020318012A1E088F070F3025
:10042000142A0F30142AFF309B009B0B152A08005A
:10043000FF309C004F309B009B0B1C2A9C0B1A2A00
:10044000080083160610831206140F2286140F224A
:1004500006100F228610080083160610831206105D
:100460000F2286140F220614080083160614831226
:1004700008309A00950D151086140F2206181514D1
:100480000F2286109A0B3A2A080083160610831250
:1004900008309A00961F4E2A06144F2A06100F2283
:1004A00086140F228610960D9A0B4A2A960D0F225B
:1004B00006140F2286140F228610080083160610D9
:1004C000831206100F2286140F228610080083164E
:1004D0000610831206140F2286140F2286100800BD
:1004E00083160610831206140F2286140F2286101C
:1004F0000F220800031083160814831208089500C1
:100500000800031016088800831608128B13553054
:100510008900AA3089008814081E8C2A08128B17BB
:1005200083120800A50083120308A6002608830092
:040530002508090091
:00000001FF
